 flexcansdk

 Timestamp is 4fb05c7c (Mon May 14 13:14:36 2012)

 Preferred load address is 10000000

 Start         Length     Name                   Class
 0001:00000000 00000004H .CRT$XCA                CODE
 0001:00000004 00000004H .CRT$XCZ                CODE
 0001:00000008 00000004H .CRT$XIA                CODE
 0001:0000000c 00000004H .CRT$XIZ                CODE
 0001:00000010 00000004H .CRT$XPA                CODE
 0001:00000014 00000004H .CRT$XPZ                CODE
 0001:00000018 00000004H .CRT$XTA                CODE
 0001:0000001c 00000004H .CRT$XTZ                CODE
 0001:00000020 0000130cH .rdata                  CODE
 0001:0000132c 00000027H .rdata$debug            CODE
 0001:00001354 000022a4H .text                   CODE
 0001:000035f8 00000034H .xdata                  CODE
 0001:0000362c 00000014H .idata$2                CODE
 0001:00003640 00000014H .idata$3                CODE
 0001:00003654 00000070H .idata$4                CODE
 0001:000036c4 0000000cH .idata$6                CODE
 0001:000036d0 000000eeH .edata                  CODE
 0002:00000000 00000070H .idata$5                DATA
 0002:00000070 0000044cH .data                   DATA
 0002:000004c0 00000fc0H .bss                    DATA
 0003:00000000 00000110H .pdata                  DATA

  Address         Publics by Value              Rva+Base       Lib:Object

 0000:00000000       ___safe_se_handler_count   00000000     <absolute>
 0000:00000000       ___safe_se_handler_table   00000000     <absolute>
 0001:00000000       __xc_a                     10001000     corelib0:crt0init.obj
 0001:00000004       __xc_z                     10001004     corelib0:crt0init.obj
 0001:00000008       __xi_a                     10001008     corelib0:crt0init.obj
 0001:0000000c       __xi_z                     1000100c     corelib0:crt0init.obj
 0001:00000010       __xp_a                     10001010     corelib0:crt0init.obj
 0001:00000014       __xp_z                     10001014     corelib0:crt0init.obj
 0001:00000018       __xt_a                     10001018     corelib0:crt0init.obj
 0001:0000001c       __xt_z                     1000101c     corelib0:crt0init.obj
 0001:00000040       ??_C@_1EC@FMPOIOMP@?$AAF?$AAl?$AAe?$AAx?$AAC?$AAA?$AAN?$AA?5?$AAS?$AAD?$AAK?$AA?3?$AA?5?$AA?9?$AAF?$AAl?$AAe?$AAx?$AAC?$AAA?$AAN?$AAI?$AAn?$AAi?$AAt?$AA?$CI?$AA?$CF?$AAs?$AA?$CJ?$AA?9?$AA?$AN?$AA?6@ 10001040     flexcansdk.obj
 0001:00000084       ??_C@_1M@HCOOECOK@?$AAF?$AAA?$AAL?$AAS?$AAE?$AA?$AA@ 10001084     flexcansdk.obj
 0001:00000090       ??_C@_19ELAAHEEL@?$AAT?$AAR?$AAU?$AAE?$AA?$AA@ 10001090     flexcansdk.obj
 0001:000000a0       ??_C@_1JK@FAGNGMOD@?$AAF?$AAl?$AAe?$AAx?$AAC?$AAA?$AAN?$AA?5?$AAS?$AAD?$AAK?$AA?3?$AA?5?$AA?5?$AAF?$AAl?$AAe?$AAx?$AAC?$AAA?$AAN?$AAI?$AAn?$AAi?$AAt?$AA?$DO?$AA?5?$AAW?$AAA?$AAR?$AAN?$AAI@ 100010a0     flexcansdk.obj
 0001:00000140       ??_C@_1II@KANMMDMI@?$AAF?$AAl?$AAe?$AAx?$AAC?$AAA?$AAN?$AA?5?$AAS?$AAD?$AAK?$AA?3?$AA?5?$AA?5?$AAF?$AAl?$AAe?$AAx?$AAC?$AAA?$AAN?$AAI?$AAn?$AAi?$AAt?$AA?$DO?$AA?5?$AAE?$AAR?$AAR?$AAO?$AAR@ 10001140     flexcansdk.obj
 0001:000001c8       ??_C@_1KM@MCLCLDNC@?$AAF?$AAl?$AAe?$AAx?$AAC?$AAA?$AAN?$AA?5?$AAS?$AAD?$AAK?$AA?3?$AA?5?$AA?5?$AAF?$AAl?$AAe?$AAx?$AAC?$AAA?$AAN?$AAI?$AAn?$AAi?$AAt?$AA?$DO?$AA?5?$AAI?$AAN?$AAF?$AAO?$AA?3@ 100011c8     flexcansdk.obj
 0001:00000274       ??_C@_1O@IFEMKBCF@?$AAC?$AAA?$AAN?$AA?$CF?$AAd?$AA?3?$AA?$AA@ 10001274     flexcansdk.obj
 0001:00000288       ??_C@_1FG@LAOBAODD@?$AAF?$AAl?$AAe?$AAx?$AAC?$AAA?$AAN?$AA?5?$AAS?$AAD?$AAK?$AA?3?$AA?5?$AA?$CL?$AAF?$AAl?$AAe?$AAx?$AAC?$AAA?$AAN?$AAI?$AAn?$AAi?$AAt?$AA?$CI?$AAd?$AAw?$AAI?$AAn?$AAd?$AAe@ 10001288     flexcansdk.obj
 0001:000002e0       ??_C@_1EG@JOMIFMEC@?$AAF?$AAl?$AAe?$AAx?$AAC?$AAA?$AAN?$AA?5?$AAS?$AAD?$AAK?$AA?3?$AA?5?$AA?9?$AAF?$AAl?$AAe?$AAx?$AAC?$AAA?$AAN?$AAD?$AAe?$AAi?$AAn?$AAi?$AAt?$AA?$CI?$AA?$CF?$AAs?$AA?$CJ?$AA?9@ 100012e0     flexcansdk.obj
 0001:00000328       ??_C@_1KC@BMHALCBI@?$AAF?$AAl?$AAe?$AAx?$AAC?$AAA?$AAN?$AA?5?$AAS?$AAD?$AAK?$AA?3?$AA?5?$AA?5?$AAF?$AAl?$AAe?$AAx?$AAC?$AAA?$AAN?$AAD?$AAe?$AAi?$AAn?$AAi?$AAt?$AA?$DO?$AA?5?$AAW?$AAA?$AAR@ 10001328     flexcansdk.obj
 0001:000003d0       ??_C@_1JG@LDPBLAD@?$AAF?$AAl?$AAe?$AAx?$AAC?$AAA?$AAN?$AA?5?$AAS?$AAD?$AAK?$AA?3?$AA?5?$AA?5?$AAF?$AAl?$AAe?$AAx?$AAC?$AAA?$AAN?$AAD?$AAe?$AAi?$AAn?$AAi?$AAt?$AA?$DO?$AA?5?$AAE?$AAR?$AAR@ 100013d0     flexcansdk.obj
 0001:00000468       ??_C@_1JC@LBALOMCL@?$AAF?$AAl?$AAe?$AAx?$AAC?$AAA?$AAN?$AA?5?$AAS?$AAD?$AAK?$AA?3?$AA?5?$AA?5?$AAF?$AAl?$AAe?$AAx?$AAC?$AAA?$AAN?$AAD?$AAe?$AAi?$AAn?$AAi?$AAt?$AA?$DO?$AA?5?$AAI?$AAN?$AAF@ 10001468     flexcansdk.obj
 0001:00000500       ??_C@_1FK@NEOHOLFK@?$AAF?$AAl?$AAe?$AAx?$AAC?$AAA?$AAN?$AA?5?$AAS?$AAD?$AAK?$AA?3?$AA?5?$AA?$CL?$AAF?$AAl?$AAe?$AAx?$AAC?$AAA?$AAN?$AAD?$AAe?$AAi?$AAn?$AAi?$AAt?$AA?$CI?$AAd?$AAw?$AAI?$AAn@ 10001500     flexcansdk.obj
 0001:00000560       ??_C@_1EO@JEANCIEO@?$AAF?$AAl?$AAe?$AAx?$AAC?$AAA?$AAN?$AA?5?$AAS?$AAD?$AAK?$AA?3?$AA?5?$AA?9?$AAF?$AAl?$AAe?$AAx?$AAC?$AAA?$AAN?$AAW?$AAr?$AAi?$AAt?$AAe?$AAF?$AAr?$AAa?$AAm?$AAe?$AA?$CI@ 10001560     flexcansdk.obj
 0001:000005b0       ??_C@_1HK@PNMLAEDB@?$AAF?$AAl?$AAe?$AAx?$AAC?$AAA?$AAN?$AA?5?$AAS?$AAD?$AAK?$AA?3?$AA?5?$AA?5?$AAF?$AAl?$AAe?$AAx?$AAC?$AAA?$AAN?$AAW?$AAr?$AAi?$AAt?$AAe?$AAF?$AAr?$AAa?$AAm?$AAe?$AA?$DO@ 100015b0     flexcansdk.obj
 0001:00000630       ??_C@_1MK@DNGKCAJB@?$AAF?$AAl?$AAe?$AAx?$AAC?$AAA?$AAN?$AA?5?$AAS?$AAD?$AAK?$AA?3?$AA?5?$AA?5?$AAF?$AAl?$AAe?$AAx?$AAC?$AAA?$AAN?$AAW?$AAr?$AAi?$AAt?$AAe?$AAF?$AAr?$AAa?$AAm?$AAe?$AA?$DO@ 10001630     flexcansdk.obj
 0001:00000700       ??_C@_1PE@LPEPPFN@?$AAF?$AAl?$AAe?$AAx?$AAC?$AAA?$AAN?$AA?5?$AAS?$AAD?$AAK?$AA?3?$AA?5?$AA?$CL?$AAF?$AAl?$AAe?$AAx?$AAC?$AAA?$AAN?$AAW?$AAr?$AAi?$AAt?$AAe?$AAF?$AAr?$AAa?$AAm?$AAe?$AA?$CI@ 10001700     flexcansdk.obj
 0001:000007f8       ??_C@_1EM@FACFIPOP@?$AAF?$AAl?$AAe?$AAx?$AAC?$AAA?$AAN?$AA?5?$AAS?$AAD?$AAK?$AA?3?$AA?5?$AA?9?$AAF?$AAl?$AAe?$AAx?$AAC?$AAA?$AAN?$AAR?$AAe?$AAa?$AAd?$AAF?$AAr?$AAa?$AAm?$AAe?$AA?$CI?$AA?$CF@ 100017f8     flexcansdk.obj
 0001:00000848       ??_C@_1HI@FNFPCPIA@?$AAF?$AAl?$AAe?$AAx?$AAC?$AAA?$AAN?$AA?5?$AAS?$AAD?$AAK?$AA?3?$AA?5?$AA?5?$AAF?$AAl?$AAe?$AAx?$AAC?$AAA?$AAN?$AAR?$AAe?$AAa?$AAd?$AAF?$AAr?$AAa?$AAm?$AAe?$AA?$DO?$AA?5@ 10001848     flexcansdk.obj
 0001:000008c0       ??_C@_1MI@NCPNIACB@?$AAF?$AAl?$AAe?$AAx?$AAC?$AAA?$AAN?$AA?5?$AAS?$AAD?$AAK?$AA?3?$AA?5?$AA?5?$AAF?$AAl?$AAe?$AAx?$AAC?$AAA?$AAN?$AAR?$AAe?$AAa?$AAd?$AAF?$AAr?$AAa?$AAm?$AAe?$AA?$DO?$AA?5@ 100018c0     flexcansdk.obj
 0001:00000988       ??_C@_1MO@DAKAIICN@?$AAF?$AAl?$AAe?$AAx?$AAC?$AAA?$AAN?$AA?5?$AAS?$AAD?$AAK?$AA?3?$AA?5?$AA?$CL?$AAF?$AAl?$AAe?$AAx?$AAC?$AAA?$AAN?$AAR?$AAe?$AAa?$AAd?$AAF?$AAr?$AAa?$AAm?$AAe?$AA?$CI?$AAd@ 10001988     flexcansdk.obj
 0001:00000a58       ??_C@_1EK@JLFPPLAP@?$AAF?$AAl?$AAe?$AAx?$AAC?$AAA?$AAN?$AA?5?$AAS?$AAD?$AAK?$AA?3?$AA?5?$AA?9?$AAF?$AAl?$AAe?$AAx?$AAC?$AAA?$AAN?$AAT?$AAr?$AAa?$AAn?$AAs?$AAf?$AAe?$AAr?$AA?$CI?$AA?$CF?$AAs@ 10001a58     flexcansdk.obj
 0001:00000aa8       ??_C@_1HG@GMHDNFJN@?$AAF?$AAl?$AAe?$AAx?$AAC?$AAA?$AAN?$AA?5?$AAS?$AAD?$AAK?$AA?3?$AA?5?$AA?5?$AAF?$AAl?$AAe?$AAx?$AAC?$AAA?$AAN?$AAT?$AAr?$AAa?$AAn?$AAs?$AAf?$AAe?$AAr?$AA?$DO?$AA?5?$AAE@ 10001aa8     flexcansdk.obj
 0001:00000b20       ??_C@_1MG@NJCKBIAO@?$AAF?$AAl?$AAe?$AAx?$AAC?$AAA?$AAN?$AA?5?$AAS?$AAD?$AAK?$AA?3?$AA?5?$AA?5?$AAF?$AAl?$AAe?$AAx?$AAC?$AAA?$AAN?$AAT?$AAr?$AAa?$AAn?$AAs?$AAf?$AAe?$AAr?$AA?$DO?$AA?5?$AAE@ 10001b20     flexcansdk.obj
 0001:00000be8       ??_C@_1JA@NHDAHGKC@?$AAF?$AAl?$AAe?$AAx?$AAC?$AAA?$AAN?$AA?5?$AAS?$AAD?$AAK?$AA?3?$AA?5?$AA?$CL?$AAF?$AAl?$AAe?$AAx?$AAC?$AAA?$AAN?$AAT?$AAr?$AAa?$AAn?$AAs?$AAf?$AAe?$AAr?$AA?$CI?$AAd?$AAw@ 10001be8     flexcansdk.obj
 0001:00000c78       ??_C@_1EA@MGBLBHEP@?$AAF?$AAl?$AAe?$AAx?$AAC?$AAA?$AAN?$AA?5?$AAS?$AAD?$AAK?$AA?3?$AA?5?$AA?9?$AAF?$AAl?$AAe?$AAx?$AAC?$AAA?$AAN?$AAS?$AAe?$AAt?$AA?$CI?$AA?$CF?$AAs?$AA?$CJ?$AA?9?$AA?$AN?$AA?6?$AA?$AA@ 10001c78     flexcansdk.obj
 0001:00000cb8       ??_C@_1GM@IFOOLDPG@?$AAF?$AAl?$AAe?$AAx?$AAC?$AAA?$AAN?$AA?5?$AAS?$AAD?$AAK?$AA?3?$AA?5?$AA?5?$AAF?$AAl?$AAe?$AAx?$AAC?$AAA?$AAN?$AAS?$AAe?$AAt?$AA?$DO?$AA?5?$AAE?$AAR?$AAR?$AAO?$AAR?$AA?3@ 10001cb8     flexcansdk.obj
 0001:00000d28       ??_C@_1LM@FFFGFKAO@?$AAF?$AAl?$AAe?$AAx?$AAC?$AAA?$AAN?$AA?5?$AAS?$AAD?$AAK?$AA?3?$AA?5?$AA?5?$AAF?$AAl?$AAe?$AAx?$AAC?$AAA?$AAN?$AAS?$AAe?$AAt?$AA?$DO?$AA?5?$AAE?$AAR?$AAR?$AAO?$AAR?$AA?3@ 10001d28     flexcansdk.obj
 0001:00000de8       ??_C@_1KA@CBKMMNGH@?$AAF?$AAl?$AAe?$AAx?$AAC?$AAA?$AAN?$AA?5?$AAS?$AAD?$AAK?$AA?3?$AA?5?$AA?$CL?$AAF?$AAl?$AAe?$AAx?$AAC?$AAA?$AAN?$AAS?$AAe?$AAt?$AA?$CI?$AAd?$AAw?$AAI?$AAn?$AAd?$AAe?$AAx@ 10001de8     flexcansdk.obj
 0001:00000e88       ??_C@_1EA@DDENMOAO@?$AAF?$AAl?$AAe?$AAx?$AAC?$AAA?$AAN?$AA?5?$AAS?$AAD?$AAK?$AA?3?$AA?5?$AA?9?$AAF?$AAl?$AAe?$AAx?$AAC?$AAA?$AAN?$AAG?$AAe?$AAt?$AA?$CI?$AA?$CF?$AAs?$AA?$CJ?$AA?9?$AA?$AN?$AA?6?$AA?$AA@ 10001e88     flexcansdk.obj
 0001:00000ec8       ??_C@_1GM@DMIFMFLN@?$AAF?$AAl?$AAe?$AAx?$AAC?$AAA?$AAN?$AA?5?$AAS?$AAD?$AAK?$AA?3?$AA?5?$AA?5?$AAF?$AAl?$AAe?$AAx?$AAC?$AAA?$AAN?$AAG?$AAe?$AAt?$AA?$DO?$AA?5?$AAE?$AAR?$AAR?$AAO?$AAR?$AA?3@ 10001ec8     flexcansdk.obj
 0001:00000f38       ??_C@_1LM@IAAIOJKC@?$AAF?$AAl?$AAe?$AAx?$AAC?$AAA?$AAN?$AA?5?$AAS?$AAD?$AAK?$AA?3?$AA?5?$AA?5?$AAF?$AAl?$AAe?$AAx?$AAC?$AAA?$AAN?$AAG?$AAe?$AAt?$AA?$DO?$AA?5?$AAE?$AAR?$AAR?$AAO?$AAR?$AA?3@ 10001f38     flexcansdk.obj
 0001:00000ff8       ??_C@_1KA@HJPPPALB@?$AAF?$AAl?$AAe?$AAx?$AAC?$AAA?$AAN?$AA?5?$AAS?$AAD?$AAK?$AA?3?$AA?5?$AA?$CL?$AAF?$AAl?$AAe?$AAx?$AAC?$AAA?$AAN?$AAG?$AAe?$AAt?$AA?$CI?$AAd?$AAw?$AAI?$AAn?$AAd?$AAe?$AAx@ 10001ff8     flexcansdk.obj
 0001:00001098       ??_C@_1EA@GAAPGFGH@?$AAF?$AAl?$AAe?$AAx?$AAC?$AAA?$AAN?$AA?5?$AAS?$AAD?$AAK?$AA?3?$AA?5?$AA?9?$AAC?$AAa?$AAl?$AAl?$AAD?$AAr?$AAi?$AAv?$AAe?$AAr?$AA?$CI?$AA?$CF?$AAs?$AA?$CJ?$AA?9?$AA?$AN?$AA?6?$AA?$AA@ 10002098     flexcansdk.obj
 0001:000010d8       ??_C@_1GM@MMFMENPF@?$AAF?$AAl?$AAe?$AAx?$AAC?$AAA?$AAN?$AA?5?$AAS?$AAD?$AAK?$AA?3?$AA?5?$AA?5?$AAC?$AAa?$AAl?$AAl?$AAD?$AAr?$AAi?$AAv?$AAe?$AAr?$AA?$DO?$AA?5?$AAE?$AAR?$AAR?$AAO?$AAR?$AA?3@ 100020d8     flexcansdk.obj
 0001:00001148       ??_C@_1LM@BFOPLEEA@?$AAF?$AAl?$AAe?$AAx?$AAC?$AAA?$AAN?$AA?5?$AAS?$AAD?$AAK?$AA?3?$AA?5?$AA?5?$AAC?$AAa?$AAl?$AAl?$AAD?$AAr?$AAi?$AAv?$AAe?$AAr?$AA?$DO?$AA?5?$AAE?$AAR?$AAR?$AAO?$AAR?$AA?3@ 10002148     flexcansdk.obj
 0001:00001208       ??_C@_1IG@PMHKNCKG@?$AAF?$AAl?$AAe?$AAx?$AAC?$AAA?$AAN?$AA?5?$AAS?$AAD?$AAK?$AA?3?$AA?5?$AA?5?$AAC?$AAa?$AAl?$AAl?$AAD?$AAr?$AAi?$AAv?$AAe?$AAr?$AA?$DO?$AA?5?$AAE?$AAR?$AAR?$AAO?$AAR?$AA?3@ 10002208     flexcansdk.obj
 0001:00001290       ??_C@_1JM@MAAJIHM@?$AAF?$AAl?$AAe?$AAx?$AAC?$AAA?$AAN?$AA?5?$AAS?$AAD?$AAK?$AA?3?$AA?5?$AA?$CL?$AAC?$AAa?$AAl?$AAl?$AAD?$AAr?$AAi?$AAv?$AAe?$AAr?$AA?$CI?$AAd?$AAw?$AAI?$AAn?$AAd?$AAe?$AAx@ 10002290     flexcansdk.obj
 0001:00001354       ?to_T@@YAPBGPBD@Z          10002354 f   DebugZones.obj
 0001:000013f4       DllMain                    100023f4 f   flexcansdk.obj
 0001:0000144c       FlexCANInit                1000244c f   flexcansdk.obj
 0001:00001720       FlexCANDeinit              10002720 f   flexcansdk.obj
 0001:00001940       FlexCANSetBitrate          10002940 f   flexcansdk.obj
 0001:00001980       FlexCANGetBitrate          10002980 f   flexcansdk.obj
 0001:000019c8       FlexCANWriteFrame          100029c8 f   flexcansdk.obj
 0001:00001c4c       FlexCANReadFrame           10002c4c f   flexcansdk.obj
 0001:00001e7c       FlexCANTransfer            10002e7c f   flexcansdk.obj
 0001:000028fc       ??$FlexCANGet@K@@YAHKHPAK@Z 100038fc f i flexcansdk.obj
 0001:00002ab4       RegisterDbgZones           10003ab4 f   coredll:COREDLL.dll
 0001:00002ac4       DisableThreadLibraryCalls  10003ac4 f   coredll:COREDLL.dll
 0001:00002ad4       GetLastError               10003ad4 f   coredll:COREDLL.dll
 0001:00002ae4       CreateFileW                10003ae4 f   coredll:COREDLL.dll
 0001:00002af4       NKDbgPrintfW               10003af4 f   coredll:COREDLL.dll
 0001:00002b04       CloseHandle                10003b04 f   coredll:COREDLL.dll
 0001:00002b14       SetLastError               10003b14 f   coredll:COREDLL.dll
 0001:00002b24       DeviceIoControl            10003b24 f   coredll:COREDLL.dll
 0001:00002b34       _DllMainCRTStartup         10003b34 f   corelib0:pegdmain.obj
 0001:00002cdc       __security_init_cookie     10003cdc f   corelib0:seccinit.obj
 0001:00002da4       __GSHandlerCheck           10003da4 f   corelib0:gshandler.obj
 0001:00002dec       __GSHandlerCheckCommon     10003dec f   corelib0:gshandler.obj
 0001:00002e94       __security_check_cookie    10003e94 f   corelib0:armsecgs.obj
 0001:00002ea8       __gsfailure                10003ea8 f   corelib0:armsecgs.obj
 0001:00002eec       exit                       10003eec f   corelib0:cexit.obj
 0001:0000306c       _exit                      1000406c f   corelib0:cexit.obj
 0001:00003090       _cexit                     10004090 f   corelib0:cexit.obj
 0001:000030ac       _c_exit                    100040ac f   corelib0:cexit.obj
 0001:000030c8       GetCurrentProcess          100040c8 f i corelib0:cexit.obj
 0001:000030e0       _initterm                  100040e0 f   corelib0:crt0dat.obj
 0001:00003134       _cinit                     10004134 f   corelib0:crt0dat.obj
 0001:00003170       _onexit                    10004170 f   corelib0:onexit.obj
 0001:00003474       atexit                     10004474 f   corelib0:onexit.obj
 0001:000034c8       mbstowcs                   100044c8 f   corelib1:COREDLL.dll
 0001:000034d8       swprintf                   100044d8 f   corelib1:COREDLL.dll
 0001:000034e8       memcpy                     100044e8 f   corelib1:COREDLL.dll
 0001:000034f8       memset                     100044f8 f   corelib1:COREDLL.dll
 0001:00003508       _XcptFilter                10004508 f   corelib1:COREDLL.dll
 0001:00003518       __C_specific_handler       10004518 f   corelib1:COREDLL.dll
 0001:00003528       __security_gen_cookie2     10004528 f   corelib1:COREDLL.dll
 0001:00003538       __report_gsfailure         10004538 f   corelib1:COREDLL.dll
 0001:00003548       free                       10004548 f   corelib1:COREDLL.dll
 0001:00003558       malloc                     10004558 f   corelib1:COREDLL.dll
 0001:00003568       realloc                    10004568 f   corelib1:COREDLL.dll
 0001:00003578       _msize                     10004578 f   corelib1:COREDLL.dll
 0001:00003588       DeleteCriticalSection      10004588 f   coredll:COREDLL.dll
 0001:00003598       InterlockedExchange        10004598 f   coredll:COREDLL.dll
 0001:000035a8       TerminateProcess           100045a8 f   coredll:COREDLL.dll
 0001:000035b8       EnterCriticalSection       100045b8 f   coredll:COREDLL.dll
 0001:000035c8       InterlockedCompareExchange 100045c8 f   coredll:COREDLL.dll
 0001:000035d8       InitializeCriticalSection  100045d8 f   coredll:COREDLL.dll
 0001:000035e8       LeaveCriticalSection       100045e8 f   coredll:COREDLL.dll
 0001:0000362c       __IMPORT_DESCRIPTOR_COREDLL 1000462c     coredll:COREDLL.dll
 0001:00003640       __NULL_IMPORT_DESCRIPTOR   10004640     coredll:COREDLL.dll
 0002:00000000       __imp_RegisterDbgZones     10005000     coredll:COREDLL.dll
 0002:00000004       __imp_DisableThreadLibraryCalls 10005004     coredll:COREDLL.dll
 0002:00000008       __imp_GetLastError         10005008     coredll:COREDLL.dll
 0002:0000000c       __imp_CreateFileW          1000500c     coredll:COREDLL.dll
 0002:00000010       __imp_NKDbgPrintfW         10005010     coredll:COREDLL.dll
 0002:00000014       __imp_CloseHandle          10005014     coredll:COREDLL.dll
 0002:00000018       __imp_SetLastError         10005018     coredll:COREDLL.dll
 0002:0000001c       __imp_DeviceIoControl      1000501c     coredll:COREDLL.dll
 0002:00000020       __imp_mbstowcs             10005020     corelib1:COREDLL.dll
 0002:00000024       __imp_swprintf             10005024     corelib1:COREDLL.dll
 0002:00000028       __imp_memcpy               10005028     corelib1:COREDLL.dll
 0002:0000002c       __imp_memset               1000502c     corelib1:COREDLL.dll
 0002:00000030       __imp__XcptFilter          10005030     corelib1:COREDLL.dll
 0002:00000034       __imp___C_specific_handler 10005034     corelib1:COREDLL.dll
 0002:00000038       __imp___security_gen_cookie2 10005038     corelib1:COREDLL.dll
 0002:0000003c       __imp___report_gsfailure   1000503c     corelib1:COREDLL.dll
 0002:00000040       __imp_free                 10005040     corelib1:COREDLL.dll
 0002:00000044       __imp_malloc               10005044     corelib1:COREDLL.dll
 0002:00000048       __imp_realloc              10005048     corelib1:COREDLL.dll
 0002:0000004c       __imp__msize               1000504c     corelib1:COREDLL.dll
 0002:00000050       __imp_DeleteCriticalSection 10005050     coredll:COREDLL.dll
 0002:00000054       __imp_InterlockedExchange  10005054     coredll:COREDLL.dll
 0002:00000058       __imp_TerminateProcess     10005058     coredll:COREDLL.dll
 0002:0000005c       __imp_EnterCriticalSection 1000505c     coredll:COREDLL.dll
 0002:00000060       __imp_InterlockedCompareExchange 10005060     coredll:COREDLL.dll
 0002:00000064       __imp_InitializeCriticalSection 10005064     coredll:COREDLL.dll
 0002:00000068       __imp_LeaveCriticalSection 10005068     coredll:COREDLL.dll
 0002:0000006c       \177COREDLL_NULL_THUNK_DATA 1000506c     coredll:COREDLL.dll
 0002:00000070       dpCurSettings              10005070     DebugZones.obj
 0002:000004b4       __security_cookie          100054b4     corelib0:seccinit.obj
 0002:000004b8       __security_cookie_complement 100054b8     corelib0:seccinit.obj
 0002:0000146c       _exitflag                  1000646c     corelib0:cexit.obj
 0002:00001470       __onexitend                10006470     <common>
 0002:00001474       __onexitbegin              10006474     <common>
 0002:00001478       g_pcsExit                  10006478     <common>
 0002:0000147c       _pRawDllMain               1000647c     <common>

 entry point at        0001:00002b34

 Static symbols

 0001:00002034       ??$FlexCANSet@K@@YAHKHPAK@Z 10003034 f   flexcansdk.obj
 0001:000021ec       ??$CallDriver@UCAN_TRANSFER_BLOCK@@@@YAHKHPAUCAN_TRANSFER_BLOCK@@W4ARGUMENTIO@@@Z 100031ec f   flexcansdk.obj
 0001:00002574       ??$CallDriver@K@@YAHKHPAKW4ARGUMENTIO@@@Z 10003574 f   flexcansdk.obj
 0001:00002b88       _DllMainCRTStartupHelper   10003b88 f   corelib0:pegdmain.obj
 0001:00002f10       doexit                     10003f10 f   corelib0:cexit.obj
 0001:000031cc       lockexit                   100041cc f   corelib0:onexit.obj
 0001:00003268       unlockexit                 10004268 f   corelib0:onexit.obj
 0001:00003294       _onexit_nolock             10004294 f   corelib0:onexit.obj
